:100000000C94B8010C94D5010C94D5010C94D50135
:100010000C94D5010C94CC040C94D5010C94D5010E
:100020000C94D5010C94D5010C94FC040C94D501CE
:100030000C94D5010C94D5010C94FB040C94FB0496
:100040000C94FA040C94D5010C94D5010C94D501B0
:100050000C94D5010C9423060C94D5010C94D50175
:100060000C94D5010C94D501467265712020562F51
:10007000487A2020416D7020005020202049202007
:1000800020442020202044542000526561642044F4
:100090006F6E652020202020202000526561646959
:1000A0006E6720454550524F4D20200046726571C5
:1000B0002020562F487A2020416D7020005646207F
:1000C0004D6F746F722044726976650A0053746FC5
:1000D00072656420202020202020202020005374DE
:1000E0006F72696E6720454550524F4D2020004584
:1000F0006E646520646572204661686E656E737417
:10010000616E676500312E31202863293230303925
:100110002D32303137206D61747A6574726F6E697B
:1001200063730000000000000000060004080D00DA
:1001300000DD0800E11100E51900E82100EC2A00CB
:10014000EF3200F13A00F44200F64A00F85200FAA9
:100150005A00FC6200FD6900FE7100FE7800FF801D
:1001600000FF8700FF8E00FE9500FE9B00FDA200B1
:10017000FCA800FAAE00F8B400F6BA00F4C000F132
:10018000C500EFCA00ECCF00E8D400E5D900E1DDFE
:1001900000DDE100D9E500D4E800CFEC00CAEF00B3
:1001A000C5F100C0F400BAF600B4F800AEFA00A839
:1001B000FC00A2FD009BFE0095FE008EFF0087FF65
:1001C000007FFF0078FE0071FE0069FD0062FC0008
:1001D0005AFA0052F8004AF60042F4003AF10032AE
:1001E000EF002AEC0021E80019E50011E10008DD2C
:1001F0000000E10800E51100E81900EC2100EF2AF9
:1002000000F13200F43A00F64200F84A00FA5200D7
:10021000FC5A00FD6200FE6900FE7100FF7800FFDD
:100220007F00FF8700FE8E00FE9500FD9B00FCA274
:1002300000FAA800F8AE00F6B400F4BA00F1C0006D
:10024000EFC500ECCA00E8CF00E5D400E1D900DD3D
:10025000DD00D9E100D4E500CFE800CAEC00C5EF2D
:1002600000C0F100BAF400B4F600AEF800A8FA003D
:10027000A2FC009BFD0095FE008EFE0087FF008023
:10028000FF0078FF0071FE0069FE0062FD005AFC6D
:100290000052FA004AF80042F6003AF40032F10047
:1002A0002AEF0021EC0019E80011E50008E1000048
:1002B000DD0000E10800E51100E81900EC2100EF85
:1002C0002A00F13200F43A00F64200F84A00FA52ED
:1002D00000FC5A00FD6200FE6900FE7100FF78001C
:1002E000FF8000FF8700FE8E00FE9500FD9B00FC56
:1002F000A200FAA800F8AE00F6B400F4BA00F1C00B
:1003000000EFC500ECCA00E8CF00E5D400E1D90059
:10031000DDDD00D9E100D4E500CFE800CAEC00C57E
:10032000EF00C0F100BAF400B4F600AEF800A8FA8D
:1003300000A2FC009BFD0095FE008EFE0087FF00E2
:1003400080FF0078FF0071FE0069FE0062FD005A28
:10035000FC0052FA004AF80042F6003AF40032F18A
:10036000002AEF0021EC0019E80011E50008E10087
:1003700011241FBECFEFD8E0DEBFCDBF11E0A0E05B
:10038000B1E0E0ECF3E102C005900D92A032B107BC
:10039000D9F721E0A0E2B1E001C01D92AC33B20771
:1003A000E1F70E942B070C94DE090C940000CF9318
:1003B000DF93DC01FB01E9011A821B821C821D8292
:1003C000198218829F838E83798768875B874A8723
:1003D0008FEF9FE7BD010E9401097D876C879F0118
:1003E000FF0F440B550B61E070E08FEF9FE70E9419
:1003F00037092E873F87488B598BDF91CF9108951E
:10040000EF92FF920F931F93CF93DF938B01FA012B
:100410009C01261B370B848595858217930784F0F2
:10042000919581959109281739076CF086819781FC
:10043000289FE001299FD00D389FD00D112405C0C1
:10044000CFEFDFE702C0C1E0D0E8C901330FAA0B4C
:10045000BB0B42815381648175819A01AB01280FE6
:10046000391F4A1F5B1F86859785A089B18982172E
:100470009307A407B5074CF482839383A483B583C1
:1004800061E070E08FEF9FE71DC0B095A09590955B
:1004900081959F4FAF4FBF4F281739074A075B071A
:1004A0004CF482839383A483B5836FEF7FEF80E066
:1004B00090E808C02283338344835583A085B185A7
:1004C0000E94650920813181201B310BA285B385F3
:1004D0002A9F70012B9FF00C3A9FF00C112411837E
:1004E00000838E01DD0F220B330BAB01BC01400FEB
:1004F000511F621F731FC701FF0CAA0BBB0B8A01A0
:100500009B01080F191F2A1F3B1FC901B80120E0DA
:1005100031E040E050E00E943709213010E8310717
:100520001FEF4107510724F421E030E84FEF5FEF60
:10053000DA01C901811520E89207A105B10524F06F
:100540008FEF9FE7A0E0B0E0DF91CF911F910F9177
:10055000FF90EF900895FC0112821382148215829D
:10056000089584B1817F84B98AB187798AB9089561
:10057000CF93C82FE82FE295EF70F0E0E45FFE4FD5
:1005800080810E94C406CF70EC2FF0E0E45FFE4F44
:100590008081CF910C94C406CF93C82F892F0E94DD
:1005A000B8028C2FCF910C94B80280E20C94C40650
:1005B000DF92EF92FF920F931F93CF93DF934AE066
:1005C00060E071E00E94780980933B01E0E0F1E097
:1005D00001900020E9F73197E050F140DE2E80E0F5
:1005E000E82E81E0F82E8701FF27EF012197802F69
:1005F0008E198D1578F4C801805091408C179D0795
:1006000019F48EE20E94C406F80181918F010E94C4
:10061000C406EDCFDF91CF911F910F91FF90EF9026
:10062000DF900895DB01FA0190911E01981710F0F8
:100630001C921AC090911E01482F50E02FEF30E01D
:10064000291B3109421753073CF080911E01880F86
:1006500080958C938FEF08C090911E01282F291B45
:100660002C9390911E01890F8083089589B1809504
:100670008770089561E080E00E94B3068EED90E0FF
:100680000E94E406F8940E94B102F999FECF6091AD
:100690001E0188E090E00E94BB09F999FECF682D09
:1006A00087E090E00E94BB09F999FECF672D86E0B4
:1006B00090E00E94BB09F999FECF60912C017091E6
:1006C0002D0184E090E00E94C909F999FECF609164
:1006D0002E0170912F0182E090E00E94C909F999E2
:1006E000FECF609130017091310180E090E00E9476
:1006F000C909F999FECF292D2C60922E78948FEF9D
:1007000099E628E1815090402040E1F700C00000C8
:1007100061E080E00E94B3068DEC90E00E94E40668
:100720008FEF99E628E1815090402040E1F700C02A
:1007300000000C943603EF92FF920F931F93CF9318
:10074000DF930E94C10689E790E00E94E4061092C0
:1007500021010E9436038111FCCFD0E088ECF82EF5
:1007600001E010E098E0E92E0E943603C82F8330A4
:1007700009F4A5C028F4813059F08230B1F006C0E8
:10078000843009F45CC0853009F49BC0D0E099C086
:10079000809121018F5F809321018091210184301C
:1007A00008F48FC0109221018CC08091210181300A
:1007B000B9F028F0823029F18330A1F182C0809114
:1007C0002C0190912D011816190624F010932D017B
:1007D00000932C0180912C0190912D01019742C032
:1007E00080912E0190912F011816190624F0109374
:1007F0002F0100932E0180912E0190912F010197DE
:100800003FC080913001909131011816190624F0F3
:1008100010933101009330018091300190913101AA
:1008200001973CC080911E01815080931E018091F0
:100830001E01883008F045C0E0921E0142C0809140
:1008400021018130A1F028F08230F9F0833059F194
:1008500038C080912C0190912D0180912C019091B4
:100860002D01019690932D0180932C012AC0809137
:100870002E0190912F0180912E0190912F010196D0
:1008800090932F0180932E011CC080913001909194
:1008900031018091300190913101019690933101A5
:1008A000809330010EC080911E018F5F80931E01E6
:1008B00080911E01893C28F0F0921E0102C00E9426
:1008C0003A03409130015091310160912E017091B5
:1008D0002F0180912C0190912D0126E231E00E94A0
:1008E000D7010E9436038823A1F0DF5FDA3050F48D
:1008F0002FEF8DEE92E0215080409040E1F700C054
:10090000000007C08FE39CE90197F1F700C00000E9
:10091000DBE061E080E00E94B30680912C019091C1
:100920002D010E94CC0280912E0190912F010E94F6
:10093000CC0280913001909131010E94CC020E9442
:10094000D50280911E010E94B8020E94D502E0915A
:100950002101F0E0E55DFE4F849161E00E94B30665
:100960008FE19EE40197F1F700C00000C53009F067
:10097000FBCE109221010E94BE0688E690E00E9404
:10098000E4060E9436038111FCCFDF91CF911F91C5
:100990000F91FF90EF9008951F920F920FB60F9254
:1009A00011242F933F934F935F936F937F938F9374
:1009B0009F93AF93BF93EF93FF9389B18095881F67
:1009C0008827881F80FB91F80E94B102892D8C60D6
:1009D000982EFF91EF91BF91AF919F918F917F9151
:1009E0006F915F914F913F912F910F900FBE0F909C
:1009F0001F901895189518951F920F920FB60F9289
:100A00001124CF92DF92EF92FF920F931F932F93B7
:100A10003F934F935F936F937F938F939F93AF9386
:100A2000BF93EF93FF93CF93DF9300D0CDB7DEB7A3
:100A3000892D869586958370813011F10E94B102CF
:100A400081EB84BD92EB909380008093B000109274
:100A5000B3001092880017BC8FEF8093B40080938E
:100A60008A0088BD80E286BBB59BFECF892D837F3F
:100A70008460982E84B18E6084B98AB188668AB900
:100A8000882D90E01C012091380130913901820FAE
:100A9000931F909339018093380180913801909190
:100AA00039018115904C48F08091380190913901BD
:100AB000905C909339018093380180913801909136
:100AC0003901892F9927FC01EE0FFF1F8E0F9F1F01
:100AD000FC01E15DFE4F8F010F5F1F4F2491CF019D
:100AE0000296F80191FC04C00491FC01E49003C05B
:100AF000E490FC010491629E900111246E9C7001AF
:100B00001124609E80011124AE014F5F5F4FBE0132
:100B10006E5F7F4F832F0E9412038A8187BD898178
:100B200088BDAE014F5F5F4FBE016E5F7F4F8F2D5F
:100B30000E9412038A8180938800898180938A00B1
:100B4000AE014F5F5F4FBE016E5F7F4F812F0E94EE
:100B500012038A818093B30089818093B4008091CD
:100B600022018F5F80932201883C08F451C090FEDF
:100B700016C020913A01C0903A01E82DF0E030E033
:100B8000AFEFB0E00E945609BB27A92F982F872FFF
:100B900046E251E0BF010E9400028C0D882E682DB4
:100BA00070E080E09BE40E94ED089B0140E050E093
:100BB00066ED7CED81E090E00E94150930932501FF
:100BC00020932401C9016AE070E00E94ED08769E3E
:100BD0009001779E300D1124B90180E090E0232B25
:100BE00059F0663FF9E07F078105910544F066EF13
:100BF00079E080E090E003C060E070E0CB012AE0A3
:100C000030E040E050E00E943709622E109222014D
:100C10000F900F90DF91CF91FF91EF91BF91AF9126
:100C20009F918F917F916F915F914F913F912F9104
:100C30001F910F91FF90EF90DF90CF900F900FBE1C
:100C40000F901F90189578941F920F920FB60F92E5
:100C500011242F938F939F9390FE22C080917C004C
:100C6000843659F08536B1F48091790090E0870D93
:100C7000911D95958795782E0DC020913A01809110
:100C8000790090E0820F911D9595879580933A01A8
:100C900085E601C084E680937C008EED80937A0027
:100CA0009F918F912F910F900FBE0F901F901895CD
:100CB000289A00C0289808951F93CF93DF931F921E
:100CC000CDB7DEB7662311F02C9A01C02C982D9871
:100CD00097B19F6097B998B1192F107F982F92956F
:100CE0009F70912B98B989830E94580689818F70D3
:100CF000812B88B90E9458061F6018B90F90DF91A8
:100D0000CF911F9108952C982D9A87B1807F87B934
:100D1000289A00C096B1289800C0289A00C026B131
:100D20002F70892F8295807F2898822B08950E94AA
:100D3000830687FDFCCF88E090E00197F1F70C94E3
:100D40008306CF93C82F0E94970660E08C2FCF9127
:100D50000C945C06CF93C82F0E94970661E08C2FFD
:100D6000CF910C945C06611102C0805801C0805480
:100D70000C94A1060E94970690E0089581E00C94DF
:100D8000A10682E00C94A106CF93C82F0E9497067B
:100D9000CA3049F4803410F080E001C080E480580B
:100DA000CF910C94A10661E08C2FCF910C945C063E
:100DB000CF93DF93EC018991882319F00E94C40638
:100DC000FACFDF91CF910895CF93DF93FC01849107
:100DD000EF012196882321F00E94C406FE01F7CF7F
:100DE000DF91CF9108951F93CF93DF93182F97B181
:100DF0009F6097B9249A259A209AE0E0FAEF3197FC
:100E0000F1F7419A409A0E945806E0E0FEE43197DB
:100E1000F1F70E945806C0E0D1E0FE013197F1F7EA
:100E20000E945806FE013197F1F740980E9458063B
:100E30002197F1F788E20E94A10688E00E94A106AE
:100E40000E94BE0686E00E94A106812FDF91CF910D
:100E50001F910C94A106F894612C10923A018824F9
:100E60008394109221018FE087B985B1817F85B984
:100E70008BB187798BB98AB1887F8AB98BB1876941
:100E80008BB98CE00E94F3060E94C1068DEB90E0C6
:100E90000E94E40680E30E94C40681E084BD92E0E3
:100EA000909380008093B0002FEF30E03093870064
:100EB0002093860016BC23E030E030938500209319
:100EC000840095E09093B20085BD91E190938100FC
:100ED0008093B10081E30E94C40680E880936D0096
:100EE00084E08093680082E30E94C40686E98093D0
:100EF0007A0080E380937E0084E680937C001092E9
:100F00007B0086EC80937A000E94B1022FEF83EC85
:100F100099E0215080409040E1F700C000008EED44
:100F200080937A0083E30E94C40626E231E040E128
:100F300050E068E070E080E690E00E94D70184E332
:100F40000E94C406E89490F8E89491F8E92DEC60CA
:100F50009E2E85E30E94C40689B18095881F88274C
:100F6000881F80FB91F84C9903C0689490F802C0E8
:100F7000E89490F887E286BB80E280936F0086E376
:100F80000E94C406FFEF29E688E1F150204080402E
:100F9000E1F700C0000061E080E00E94B3068BE949
:100FA00090E00E94E40688E090E00E94AD09809302
:100FB0001E0180911E01883018F488E080931E0184
:100FC00087E090E00E94AD09882E86E090E00E94C4
:100FD000AD09782E84E090E00E94B50990932D0130
:100FE00080932C0182E090E00E94B50990932F013C
:100FF00080932E0180E090E00E94B509909331012A
:10100000809330019FEFE9E6F8E19150E040F04035
:10101000E1F700C0000061E080E00E94B3068AE8CA
:1010200090E00E94E4062FEF89E698E1215080408D
:101030009040E1F700C000000E94360387E30E9461
:10104000C4060E94BE068EE00E94A1068CEA90E0D3
:101050000E94E40678940BE0CFEFD0E00E943603C4
:1010600090FC3FC08230A9F018F4813031F03EC0CE
:101070008330C9F1843001F139C0809121018F5F43
:101080008093210180912101823090F11092210101
:101090002FC080912101882319F0813039F028C0B8
:1010A000811002C0882483948A9422C0711002C0E7
:1010B000772473947A941CC080912101882319F0BD
:1010C000813041F015C0EFEF8E1202C02EEF822E5C
:1010D00083940EC0FFEF7F1202C09EEF792E7394AF
:1010E00007C0833019F40E949B0302C010922301B1
:1010F0000E9436038823C9F0809123018F5F80937B
:1011000023018A3050F42FEF8DEE92E02150804081
:101110009040E1F700C0000008C0EFE3FCE9319720
:10112000F1F700C000000093230161E080E00E941D
:10113000B30680912401909125010E94D8020E945B
:10114000D50261E086E00E94B306872D90E00E9400
:10115000D8020E94D5020E94D50261E08CE00E9474
:10116000B306F4E66F9EC0011124BE010E94ED0893
:10117000CB014AE060E071E00E94780980933B0176
:10118000E0E0F1E001900020E9F73197E050F14014
:101190001E2F80E0E82E81E0F82E67018C2D8E193D
:1011A000811730F4F60181916F010E94C406F6CFD9
:1011B00085E20E94C4060E94D502E0912101F0E080
:1011C000E75DFE4F849161E00E94B3068FE19EE4EB
:1011D0000197F1F700C0000041CFAA1BBB1B51E1F2
:1011E00007C0AA1FBB1FA617B70710F0A61BB70B97
:1011F000881F991F5A95A9F780959095BC01CD013C
:10120000089597FB072E16F4009407D077FD09D0B8
:101210000E94ED0807FC05D03EF4909581959F4F04
:101220000895709561957F4F0895A1E21A2EAA1B2B
:10123000BB1BFD010DC0AA1FBB1FEE1FFF1FA21786
:10124000B307E407F50720F0A21BB30BE40BF50B83
:10125000661F771F881F991F1A9469F7609570950C
:10126000809590959B01AC01BD01CF010895052E9D
:1012700097FB1EF400940E944E0957FD07D00E9470
:10128000150907FC03D04EF40C944E095095409577
:10129000309521953F4F4F4F5F4F08959095809522
:1012A000709561957F4F8F4F9F4F0895A29FB0011A
:1012B000B39FC001A39F700D811D1124911DB29F8A
:1012C000700D811D1124911D0895B7FF0C946D09B7
:1012D0000E946D09821B930B08950E945609A59FD9
:1012E000900DB49F900DA49F800D911D1124089521
:1012F000BB274A3031F4992322F4BDE290958195C1
:101300009F4F0C948409BB27FB015527AA27880F00
:10131000991FAA1FA41710F0A41B83955051B9F769
:10132000A05DAA3308F0A95DA193009779F7B111E8
:10133000B1931192CB010C949D09DC01FC01672F44
:1013400071917723E1F7329704C07C916D9370839C
:101350006291AE17BF07C8F30895F999FECF92BD09
:1013600081BDF89A992780B50895A8E1B0E042E0E0
:1013700050E00C94D009262FF999FECF1FBA92BDE8
:1013800081BD20BD0FB6F894FA9AF99A0FBE019666
:1013900008950E94BB09272F0C94BC09DC01CB01E6
:1013A000FC01F999FECF06C0F2BDE1BDF89A319675
:1013B00000B40D9241505040B8F70895F894FFCF13
:1013C0003030303030303030303030303031323317
:1013D000343536373839414243444546000014001D
:00000001FF
